S00C0000555453322E73726563EA
S113000087C20000A6C20000A4C20000A2C2000071
S1130010A0C200009EC200009CC200009AC2000060
S113002098C2000096C2000094C2000092C2000070
S113003090C200008EC200008CC200008AC2000080
S113004088C2000086C2000084C2000082C2000090
S113005080C200007EC200007CC200007AC20000A0
S113006078C2000076C2000074C2000072C20000B0
S113007070C200006EC200006CC200006AC20000C0
S113008068C2000066C2000064C2000062C20000D0
S113009060C200005EC200005CC200000C94050A4D
S11300A00C94370A0C94690A0C949B0A52C20000FF
S11300B050C200004EC200004CC200004AC2000000
S11300C048C2000046C2000044C2000042C2000010
S11300D040C200003EC200003CC200003AC2000020
S11300E038C2000036C2000034C2000032C2000030
S11300F030C200002EC200002CC200002AC2000040
S113010028C2000026C2000024C2000022C200004F
S113011020C200001EC200001CC200000C943D0955
S11301200C946F090C94A1090C94D30912C2000019
S113013010C200000EC200000CC200000AC200007F
S113014008C2000006C2000004C2000002C200008F
S113015000C20000FEC10000FCC10000FAC10000A2
S1130160F8C10000F6C10000F4C10000F2C10000B3
S1130170F0C10000EEC10000ECC10000EAC10000C3
S1130180E8C10000E6C10000E4C10000E2C10000D3
S1130190E0C10000DEC10000DCC10000DAC10000E3
S11301A0D8C10000D6C10000D4C10000D2C10000F3
S11301B0D0C10000CEC10000CCC10000CAC1000003
S11301C0C8C10000C6C10000C4C10000C2C1000013
S11301D0C0C10000BEC10000BCC10000BAC1000023
S11301E0B8C10000B6C10000B4C10000B2C1000033
S11301F0B0C10000AEC10000ACC1000008000000A6
S1130200BE922449123EABAAAA2ABECDCCCC4C3E07
S113021000000080BEABAAAAAA3E00000000BF00F6
S11302200000803F0000000000084178D3BB4387F2
S1130230D1133D190E3CC3BD4282AD2B3E68EC8206
S113024076BED98FE1A93E4C80EFFFBE01C4FF7F8B
S11302503F000000000007634236B79BD8A71A3955
S1130260685618AEBAAB558C1D3CB7CC5763BD6D00
S1130270EDFD753EF6177231BF000000803F0000AF
S113028000000000002020202020002050505000BA
S11302900000005050F850F850502078A07028F01A
S11302A020C0C810204098186090A040A8906860B2
S11302B0204000000000102040404020104020104A
S11302C010102040005020F8205000002020F8207A
S11302D0200000000000602040000000F800000042
S11302E0000000000060600008102040800070885A
S11302F098A8C8887020602020202070708808107A
S11303002040F8F810201008887010305090F81031
S113031010F880F008088870304080F0888870F801
S113032008102040404070888870888870708888E1
S11303307808106000606000606000006060006029
S11303402040081020402010080000F800F80000A9
S11303508040201020408070880810200020708881
S11303600868A8A87070888888F88888F08888F059
S11303708888F070888080808870E0908888889071
S1130380E0F88080F08080F8F88080E080808070E1
S1130390888080988870888888F888888870202069
S11303A020202070381010101090608890A0C0A0F9
S11303B09088808080808080F888D8A88888888801
S11303C08888C8A898888870888888888870F08801
S11303D088F080808070888888A89068F08888F089
S11303E0A09088788080700808F0F82020202020D1
S11303F02088888888888870888888888850208899
S11304008888A8A8D88888885020508888888850E8
S113041020202020F80810204080F83820202020B8
S1130420203800804020100800E02020202020E018
S113043020508800000000000000000000F8402068
S11304401000000000000070087888788080B0C830
S11304508888F00000708080887008086898888810
S11304607800007088F88070304840E040404000D8
S11304700078887808308080B0C888888820006038
S113048020202070100030101090604040485060D0
S11304905048602020202020700000D0A8A8888820
S11304A00000B0C8888888000070888888700000C0
S11304B0F088F08080000068987808080000B0C8D0
S11304C0808080000070807008F04040E040404828
S11304D03000008888889868000088888850200048
S11304E0008888A8A8500000885020508800008800
S11304F0887808700000F8102040F8102020402070
S113050020102020202020202040202010202040C7
S113051011241FBECFEFCDBFDFE5DEBF00E00CBF6F
S113052010E2A0E0B0E2E4EEFDE200E00BBF02C0A6
S113053007900D92A636B107D9F722E2A6E6B0E2FB
S113054001C01D92AC3FB207E1F70E94AF0F0C94BB
S1130550F01656CDCF93DF931F921F92CDB7DEB71F
S1130560613069F5809167208F5F809367208130C7
S113057039F4409368205093692010926C2014C081
S11305802091682030916920420F531F569547955A
S11305904093682050936920843031F4109267208E
S11305A081E080936C2039C08FB78A83F8949A8154
S11305B0E0E0F2E08081846080839FBF2EC06230DF
S11305C061F5809166208F5F80936620813039F4D5
S11305D040936A2050936B2010926D2014C0209198
S11305E06A2030916B20420F531F569547954093D4
S11305F06A2050936B20843031F41092662081E09D
S113060080936D200AC08FB78983F8949981E0E0C4
S1130610F2E08081886080839FBF0F900F90DF910C
S1130620CF910895CF93DF931F92CDB7DEB78FB7E5
S11306308983F894998180916D20882321F0109208
S11306406D209FBF01C09FBF0F90DF91CF91089590
S11306501F93CF93DF93CDB7DEB72B97CDBFDEBF0C
S1130660BE016F5F7F4F80E092E0FDD7AE01485F2F
S11306705F4F61E080E092E00E94B70B8A819B812A
S11306809F7890619B8392E09D83817E80618A83C1
S11306901C82BE016F5F7F4F80E092E07ED76AEAE2
S11306A072E080E092E04BD311E0188719868A85C6
S11306B0807F81608A87AE01485F5F4F61E080E0A0
S11306C092E00E946C0B188788E08987AE01485F2E
S11306D05F4F62E080E092E0FFD780E092E08BD34E
S11306E02B96CDBFDEBFDF91CF911F910895CF939D
S11306F0DF93C0916A20D0916B20BE0180E090E02E
S11307000E949B11C53AD14080F021E836E242E4D0
S11307105DEB0E946E1223E333E345E552E40E944D
S11307209E100E946A11862F0FC02DE231E24FE91C
S11307305DEB0E946E1223E333E342E852E40E942D
S11307409E100E946A11862FDF91CF91089504C0F4
S1130750615071098109910961157105810591053E
S1130760B9F70895BF92CF92DF92EF92FF920F9361
S11307701F93CF93DF931F92CDB7DEB700E016E04F
S11307806894FF24F3F8F801F68264E070E080E0F6
S113079090E0DDDFF801F58264E070E080E090E055
S11307A0D6DF0F2EFBE2BF2EF02DB98280EA99E04E
S11307B00E94020CC12CD12C760100E412E42FE03B
S11307C030E043E0BE016F5F7F4F80EA99E00E9412
S11307D0310C00E616E0FF24F394F801F682B982A6
S11307E0BE016F5F7F4F80EA99E00E944B0CF801D5
S11307F0F682E0EAF9E0818185FFFDCF80EA80930B
S1130800A009E0EAF9E0818186FFFDCFE0EAF9E0A2
S113081080E481838081BE016F5F7F4F80EA99E02D
S11308200E94610C8BE28983BE016F5F7F4F80EA77
S113083099E00E944B0C81E080936606E0EAF9E0BF
S1130840818185FFFDCF86EA8093A009E0EAF9E083
S1130850818186FFFDCFE0EAF9E080E48183808135
S1130860BE016F5F7F4F80EA99E00E94610C8BE2CA
S11308708983BE016F5F7F4F80EA99E00E944B0C31
S113088081E080936606E0EAF9E0818185FFFDCF8F
S113089088EC8093A009E0EAF9E0818186FFFDCF2E
S11308A0E0EAF9E080E481838081BE016F5F7F4FDD
S11308B080EA99E00E94610C8BE28983BE016F5F3C
S11308C07F4F80EA99E0E7D781E080936606E0EA0B
S11308D0F9E0818185FFFDCF82EA8093A009E0EAF7
S11308E0F9E0818186FFFDCFE0EAF9E080E48183CD
S11308F08081BE016F5F7F4F80EA99E0E2D78BE28F
S11309008983BE016F5F7F4F80EA99E0C4D781E09D
S113091080936606E0EAF9E0818185FFFDCF8FE2EE
S11309208093A009E0EAF9E0818186FFFDCFE0EA47
S1130930F9E080E481838081BE016F5F7F4F80EAAC
S113094099E0BFD78BE28983BE016F5F7F4F80EA56
S113095099E0A1D781E080936606E0EAF9E081811D
S113096085FFFDCF88EF8093A009E0EAF9E081815B
S113097086FFFDCFE0EAF9E080E481838081BE0157
S11309806F5F7F4F80EA99E09CD78BE28983BE0139
S11309906F5F7F4F80EA99E07ED781E0809366069F
S11309A0E0EAF9E0818185FFFDCF1092A009E0EA39
S11309B0F9E0818186FFFDCFE0EAF9E080E48183FC
S11309C08081BE016F5F7F4F80EA99E07AD78BE226
S11309D08983BE016F5F7F4F80EA99E05CD781E035
S11309E080936606E0EAF9E0818185FFFDCF81E22C
S11309F08093A009E0EAF9E0818186FFFDCFE0EA77
S1130A00F9E080E481838081BE016F5F7F4F80EADB
S1130A1099E057D78BE28983BE016F5F7F4F80EAED
S1130A2099E039D781E080936606E0EAF9E08181B4
S1130A3085FFFDCF81E88093A009E0EAF9E0818198
S1130A4086FFFDCFE0EAF9E080E481838081BE0186
S1130A506F5F7F4F80EA99E034D78BE28983BE01D0
S1130A606F5F7F4F80EA99E016D781E08093660636
S1130A70E0EAF9E0818185FFFDCF81E28093A0095E
S1130A80E0EAF9E0818186FFFDCFE0EAF9E080E465
S1130A9081838081BE016F5F7F4F80EA99E011D727
S1130AA08BE28983BE016F5F7F4F80EA99E0F3D6C2
S1130AB081E080936606E0EAF9E0818185FFFDCF5D
S1130AC08FEA8093A009E0EAF9E0818186FFFDCFF7
S1130AD0E0EAF9E080E481838081BE016F5F7F4FAB
S1130AE080EA99E0EED60F90DF91CF911F910F919C
S1130AF0FF90EF90DF90CF90BF900895FF920F93F7
S1130B001F93CF93DF931F92CDB7DEB7082FF62E36
S1130B10142FF2D60F70006B8BE28983BE016F5FD6
S1130B207F4F80EA99E0B7D681E080936606E0EAD9
S1130B30F9E0918195FFFDCF0093A009E0EAF9E087
S1130B40818186FFFDCFE0EAF9E080E48183808142
S1130B50BE016F5F7F4F80EA99E0B3D60F2D0F7708
S1130B6002950F7000618BE28983BE016F5F7F4F36
S1130B7080EA99E090D681E080936606E0EAF9E0A5
S1130B80818185FFFDCF0093A009E0EAF9E081812E
S1130B9086FFFDCFE0EAF9E080E481838081BE0135
S1130BA06F5F7F4F80EA99E08CD60F2D0F708BE238
S1130BB08983BE016F5F7F4F80EA99E06CD681E044
S1130BC080936606E0EAF9E0818185FFFDCF00931A
S1130BD0A009E0EAF9E0818186FFFDCFE0EAF9E0CF
S1130BE080E481838081BE016F5F7F4F80EA99E05A
S1130BF068D68BE28983BE016F5F7F4F80EA99E0FC
S1130C004AD681E080936506E0EAF9E0818185FFB8
S1130C10FDCF1093A009E0EAF9E0818186FFFDCFC2
S1130C20E0EAF9E080E48183808181E080936606D4
S1130C30BE016F5F7F4F80EA99E043D60F90DF914A
S1130C40CF911F910F91FF9008950F931F93CF930E
S1130C50DF931F92CDB7DEB78EE690E248D682DDF1
S1130C608BE28983BE016F5F7F4F80EA99E013D6E0
S1130C7081E080936606E0EAF9E0818185FFFDCF9B
S1130C8080E48093A009E0EAF9E0818186FFFDCF4A
S1130C90E0EAF9E080E481838081BE016F5F7F4FE9
S1130CA080EA99E00ED600E00AC040E0612F802F70
S1130CB025DF1F5F1038C9F70F5F043011F010E013
S1130CC0F4CF0F90DF91CF911F910F910895FF9270
S1130CD00F931F93CF93DF9388234CF1603238F541
S1130CE0D42FC82FF62EF694F694F69470E088E08C
S1130CF0F89E60197109112481E090E08C0102C012
S1130D00000F111F6A95E2F76C2F8F2D03D6D13097
S1130D1021F028F0D23031F006C0802B04C00095B9
S1130D20802301C08027482F6C2F8F2DE7DEDF91B1
S1130D30CF911F910F91FF900895ECC50895CF9323
S1130D40DF931F92CDB7DEB72FB72983F89449817B
S1130D50282F392F211582E0380729F46093F422D3
S1130D607093F52207C02034324021F46093F222BC
S1130D707093F3224FBF0F90DF91CF9108958115A7
S1130D8022E0920761F480916F2291E0980F909392
S1130D906F22811112C062E081E046C6089580345A
S1130DA0924059F480916E2291E0980F90936E22B4
S1130DB0811103C062E082E037C60895811522E004
S1130DC0920759F480916F22815080936F22811190
S1130DD011C062E081E03EC608958034924051F42F
S1130DE080916E22815080936E22811103C062E053
S1130DF082E030C60895EF92FF921F93CF93DF9362
S1130E001F921F92CDB7DEB77C018FB78983F89408
S1130E101981C701B4DFF7018081816080831FBF1E
S1130E208091F7228F3F09F4FFCF8FB78A83F8941C
S1130E309A81E6EFF2E281818F5F81839FBF0F90F9
S1130E400F90DF91CF911F91FF90EF900895CF9273
S1130E50DF92EF92FF920F931F93CF93DF93EC01F6
S1130E60D901C801B695A79597958795481759074D
S1130E706A077B0778F46A017B01CC0CDD1CEE1C4D
S1130E80FF1CC901B801A70196010E94F11321506A
S1130E90310902C020E030E0832F8F708F832E83CE
S1130EA0DF91CF911F910F91FF90EF90DF90CF9042
S1130EB00895DF92EF92FF920F931F93CF93DF93E6
S1130EC01F92CDB7DEB77C018B01009709F4B2C144
S1130ED0803C910521F460E180E0A6D5ABC180E8B7
S1130EE0E81681E0F80621F462E080E09DD5A2C115
S1130EF0E114E1E0FE0621F461E080E095D59AC1B9
S1130F00F0E8EF16F3E0FF0621F461E081E08CD510
S1130F1091C130E9E31633E0F30621F461E082E0A5
S1130F2083D588C1E11482E0F80621F462E081E00F
S1130F307BD580C1E0E4EE16E2E0FE0621F462E037
S1130F4082E072D577C1F0E2EF16F3E0FF0621F4F8
S1130F5064E082E069D56EC1E11438E0F30621F45F
S1130F6061E083E061D566C1E11489E0F80621F40B
S1130F7061E084E059D55EC1E114EAE0FE0621F4A3
S1130F8061E085E051D556C1E114FBE0FF0621F490
S1130F9061E086E049D54EC130E4E31638E0F3065B
S1130FA021F462E083E040D545C180E4E81689E09D
S1130FB0F80621F462E084E037D53CC1E0E4EE16A3
S1130FC0EAE0FE0621F462E085E02ED533C1F0E9C3
S1130FD0EF16F8E0FF0621F464E083E025D52AC18A
S1130FE030E9E31639E0F30621F464E084E01CD52B
S1130FF021C180E9E8168AE0F80621F464E085E07E
S113100013D518C1E0E9EE16EBE0FE0621F464E026
S113101086E00AD50FC1F0ECEF16F8E0FF0621F4E4
S113102068E083E001D506C130ECE31639E0F3064D
S113103021F468E084E0F8D4FDC080EAE81688E092
S1131040F80661F460E183E0EFD4E0EAF8E084813B
S11310508F7E8483F801248122504CC0F0EAEF167D
S1131060F9E0FF0621F460E184E0DED4E3C030EA75
S1131070E3163AE0F30621F460E185E0D5D4DAC062
S113108080EAE8168BE0F80621F460E186E0CCD42F
S1131090D1C0E0EBEE16E8E0FE0621F460E283E066
S11310A0C3D4C8C0F0EBEF16F9E0FF0621F460E208
S11310B084E0BAD4BFC030E8E31634E0F30621F488
S11310C060E483E0B1D4B6C080EAE81684E0F806B0
S11310D021F460E485E0A8D4ADC0F70184818F7E5B
S11310E08483FB0124812250C701F0EAEF16F8E063
S11310F0FF0649F480914E0684FDA5C00F2EF1E150
S1131100DF2EF02DA4C0803B38E0930791F0803AA5
S1131110E9E09E0749F430916E0634FD9BC00F2E22
S1131120F9E1DF2EF02D16C0803BF9E09F07F1F0C6
S113113004C00F2EF5E1DF2EF02D803A3AE093073C
S113114049F480918E0684FD8AC00F2EF1E2DF2ED1
S1131150F02D15C0803A9B4091F48091AE0684FD39
S11311600AC00F2EF9E2DF2EF02D09C00F2EFDE18B
S1131170DF2EF02D04C00F2EFDE2DF2EF02DED2D1D
S1131180E695E695E69530E2E39FF0011124FA5FD7
S11311903D2D377081E090E0032E02C0880F991F27
S11311A00A94E2F78183223010F040E001C040E469
S11311B0DF015096A30FB11D9FB79983F89439812D
S11311C02C9127702C939C91942B9C933FBF8583E7
S11311D0F7018581806C8583F80184818D7F81305E
S11311E029F4F70185818260858304C0F701858134
S11311F08D7F8583F8018581882329F0F701858116
S11312008460858304C0F70185818B7F8583F80121
S1131210408151816281738100E814E82EE130E05D
S1131220C70115DEF701848188608483848180612D
S113123084831AC0F70184818F7E8483F80124811A
S11312402250C70160CF0F2EF5E1DF2EF02D80EA8A
S113125098E06ACF0F2EFDE1DF2EF02D7BCF0F2E0D
S1131260F5E2DF2EF02D8BCF0F90DF91CF911F9100
S11312700F91FF90EF90DF9008951F920F920FB699
S11312800F9211240BB60F922F933F934F935F93BA
S11312906F937F938F939F93AF93BF93EF93FF933A
S11312A04091240250912502E091F422F091F5221C
S11312B061E080E092E01995FF91EF91BF91AF91C9
S11312C09F918F917F916F915F914F913F912F915A
S11312D00F900BBE0F900FBE0F901F9018951F928A
S11312E00F920FB60F9211240BB60F922F933F93C8
S11312F04F935F936F937F938F939F93AF93BF931A
S1131300EF93FF9340912C0250912D02E091F4222F
S1131310F091F52262E080E092E01995FF91EF915F
S1131320BF91AF919F918F917F916F915F914F91F9
S11313303F912F910F900BBE0F900FBE0F901F90F7
S113134018951F920F920FB60F9211240BB60F929D
S11313502F933F934F935F936F937F938F939F93B9
S1131360AF93BF93EF93FF934091340250913502B2
S1131370E091F422F091F52264E080E092E0199586
S1131380FF91EF91BF91AF919F918F917F916F9159
S11313905F914F913F912F910F900BBE0F900FBE15
S11313A00F901F9018951F920F920FB60F92112451
S11313B00BB60F922F933F934F935F936F937F934B
S11313C08F939F93AF93BF93EF93FF9340913C020E
S11313D050913D02E091F422F091F52268E080E022
S11313E092E01995FF91EF91BF91AF919F918F91E9
S11313F07F916F915F914F913F912F910F900BBE11
S11314000F900FBE0F901F9018951F920F920FB65A
S11314100F9211240BB60F922F933F934F935F9328
S11314206F937F938F939F93AF93BF93EF93FF93A8
S11314304091640250916502E091F222F091F3220E
S113144061E080E492E01995FF91EF91BF91AF9133
S11314509F918F917F916F915F914F913F912F91C8
S11314600F900BBE0F900FBE0F901F9018951F92F8
S11314700F920FB60F9211240BB60F922F933F9336
S11314804F935F936F937F938F939F93AF93BF9388
S1131490EF93FF9340916C0250916D02E091F22220
S11314A0F091F32262E080E492E01995FF91EF91CC
S11314B0BF91AF919F918F917F916F915F914F9168
S11314C03F912F910F900BBE0F900FBE0F901F9066
S11314D018951F920F920FB60F9211240BB60F920C
S11314E02F933F934F935F936F937F938F939F9328
S11314F0AF93BF93EF93FF934091740250917502A1
S1131500E091F222F091F32264E080E492E01995F4
S1131510FF91EF91BF91AF919F918F917F916F91C7
S11315205F914F913F912F910F900BBE0F900FBE83
S11315300F901F9018951F920F920FB60F921124BF
S11315400BB60F922F933F934F935F936F937F93B9
S11315508F939F93AF93BF93EF93FF9340917C023C
S113156050917D02E091F222F091F32268E080E450
S113157092E01995FF91EF91BF91AF919F918F9157
S11315807F916F915F914F913F912F910F900BBE7F
S11315900F900FBE0F901F901895BF92CF92DF92BD
S11315A0EF92FF920F931F93CF93DF931F92CDB7C8
S11315B0DEB78C017B01811522E0920771F461E2B0
S11315C070E082E05CD2C82ED12C60E270E082E050
S11315D056D2DC2CCC24C82A10C080349240C1F5E9
S11315E065E270E082E04BD2C82ED12C64E270E058
S11315F082E045D2DC2CCC24C82A8FB78983F894A6
S1131600B980C801BCDBF801808192E09083C48674
S1131610D586F70125813681F801208F318FF701B6
S11316209281F8019283F7019481F8019483F70180
S11316309381F8019383F7019181F801918381707B
S1131640F7019081892BF8018083C801B7DBBFBE05
S11316500F90DF91CF911F910F91FF90EF90DF904A
S1131660CF90BF900895DF92EF92FF920F931F9354
S1131670CF93DF931F92CDB7DEB78C017B018FB779
S11316808983F894D980C8017ADBF8018081807C51
S1131690F7018083F801808D918DF701858396830E
S11316A0F8018281F7018283F8018481F701848340
S11316B0F8018381F7018383F8018181F701818334
S11316C0C8017CDBDFBE0F90DF91CF911F910F919A
S11316D0FF90EF90DF900895AF92BF92CF92DF9288
S11316E0EF92FF920F931F93CF93DF931F92CDB787
S11316F0DEB76C01B62E7A01862F837029F4962FFB
S11317009695969582E002C0962F80E090FF8F5FB9
S11317108601005E1F4F98E0899F000D111D112462
S11317208FB78983F894A980C60129DBF7018081EA
S1131730F8018083F7018281F8018283F7018181B6
S1131740F8018183B0FE04C0F7018381F801868328
S1131750C60134DBAFBE0F90DF91CF911F910F9183
S1131760FF90EF90DF90CF90BF90AF900895AF922D
S1131770BF92CF92DF92EF92FF920F931F93CF937A
S1131780DF931F92CDB7DEB76C01B62E7A01862F98
S1131790837029F4962F9695969582E002C0962F31
S11317A080E090FF8F5F8601005E1F4F98E0899F65
S11317B0000D111D11248FB78983F894A980C601E7
S11317C0DEDAF8018081F7018083F8018281F70174
S11317D08283F8018181F7018183B0FE04C0F8019E
S11317E08681F7018383C601E9DAAFBE0F90DF91EA
S11317F0CF911F910F91FF90EF90DF90CF90BF900A
S1131800AF900895803A28E0920721F460E183E0E4
S11318100BC10895803B28E0920721F460E283E045
S113182003C10895803A29E0920721F460E184E03D
S1131830FBC00895803B29E0920721F460E284E034
S1131840F3C00895803A2AE0920721F460E185E02C
S1131850EBC00895803A9B4019F460E186E0E4C04F
S113186008950F931F93CF93DF9300D000D0CDB78B
S1131870DEB709831A832B833C834D831E82BE010A
S11318806F5F7F4F16DB2696CDBFDEBFDF91CF9112
S11318901F910F910895FB018081E82FE695E6954D
S11318A0E69540E2E49FF0011124FA5F877021E09D
S11318B030E0A90102C0440F551F8A95E2F7468320
S11318C00895FB018081E82FE695E695E69540E2D0
S11318D0E49FF0011124FA5F877021E030E0A90150
S11318E002C0440F551F8A95E2F7458308958093FB
S11318F07022909371220895209170223091712268
S113190090E8899F200D311D1124F901E60FF11D86
S113191040830895209170223091712290E8899F2C
S1131920200D311D1124F901E60FF11D8081089568
S1131930FF920F931F93CF93DF93E42FF0E0E80F10
S1131940F11DE138F1051CF0C0E84C2F481B44237D
S113195009F44AC0D62FD695D695D69570E098E06E
S1131960D99F601971091124E1E0F0E0DF0102C0A0
S1131970AA0FBB1F6A95E2F7FA2E213021F098F0E6
S1131980223019F131C0C42F1FEF180F012F0C0F93
S1131990602F8D2FD2D94F2D482B602F8D2FAED88D
S11319A0C150A1F721C0C42F1FEF180FFA2EF094D5
S11319B0012F0C0F602F8D2FC0D94F2D4823602F7E
S11319C08D2F9CD8C150A1F70FC0C42F1FEF180F43
S11319D0012F0C0F602F8D2FB0D94F2D4827602F6A
S11319E08D2F8CD8C150A1F7DF91CF911F910F910A
S11319F0FF900895FF920F931F93CF93DF932223B9
S1131A0069F0F42E182FC22FDFEFD60F6D2F6C0F55
S1131A10202F4F2D812F8CDFC150C1F7DF91CF9143
S1131A201F910F91FF900895CF93DF931F92CDB72D
S1131A30DEB79FB79983F8949981E82FF0E0E059D5
S1131A40FF4F60958081682360839FBF0F90DF9173
S1131A50CF910895CF93DF931F92CDB7DEB79FB791
S1131A609983F8949981E82FF0E0E059FF4F808141
S1131A70682B60839FBF0F90DF91CF9108954091B1
S1131A80CA01E62FF72F8093CA0184914093CA01BB
S1131A900895AF92BF92CF92DF92EF92FF920F938D
S1131AA01F93CF93DF93C82FE62EB42E690100E075
S1131AB0F901248143816B2D8E2D9CDFF6018081F9
S1131AC0811139C08381282F269526952695877004
S1131AD009F02F5FF601A4808C2F90E03581831BE1
S1131AE091092A9D90011124829FA001839F500D8A
S1131AF0929F500D112401811281040F151FF601CC
S1131B00F380FF20A1F0D0E0C0E08E2D8C0F9C2F3D
S1131B10977021F4F801D4910F5F1F4FDD231CF45B
S1131B2041E06B2DD4D8DD0FCF5FFC12EECFB39420
S1131B30AA94A110E4CFDF91CF911F910F91FF9050
S1131B40EF90DF90CF90BF90AF900895DF92EF9227
S1131B50FF920F931F93CF93DF93D62E042F790117
S1131B60EC01162F89918A3031F4F70184818F5F5B
S1131B70080F1D2D09C08D3039F09701402F612FBA
S1131B8088DFF7018381180F88818111EBCFDF9102
S1131B90CF911F910F91FF90EF90DF900895CF9315
S1131BA0DF93FC0120E030E0C62FD0E0DE01022EFE
S1131BB002C0B595A7950A94E2F7A0FD508B2F5F5C
S1131BC03F4F31962830310589F740FF0AC041FF65
S1131BD003C0FC01658302C0FC016683FC016183D0
S1131BE002C0FC016283DF91CF91089543E050E08D
S1131BF061E080EE97E0D3DF43E050E062E080EE06
S1131C0097E0CDDF43E050E060E180E696E0C7DF97
S1131C1041E050E460E280E696E0C1DF40E05BE151
S1131C2060E280E896E0BBDF40E05BE162E080EAEE
S1131C3096E0B5DF40E05BE164E080EA96E0AFDF88
S1131C4043E050E062E080E696E0A9DF43E050E044
S1131C5068E080E696E0A3DF43E050E068E080EAD5
S1131C6096E09DDF43E050E061E080E696E097DF98
S1131C7043E050E068E080E096E091DF41E050E02E
S1131C8060E180E896E08BDF43E050E062E080E6CC
S1131C9096E085DF43E050E068E080E696E07FDF91
S1131CA040E050E064E080E696E079DF43E050E015
S1131CB060E180EA96E073DF40E050E061E080E0BC
S1131CC096E06DDF40E050E064E080E096E067DF9E
S1131CD040E050E062E080E296E061DF43E050E003
S1131CE068E080E496E05BDF40E050E064E080E49C
S1131CF096E055DF43E050E068E080E696E04FDF91
S1131D0040E050E064E080E696E049DF43E050E0E4
S1131D1068E080E896E043DF40E050E064E080E87B
S1131D2096E03DCF089504C061507109810991097D
S1131D306115710581059105B9F70895CF93DF9376
S1131D401F92CDB7DEB78FB78983F8949981E0E409
S1131D50F2E08081846080839FBF84A195A10F906D
S1131D60DF91CF910895161617064CF481E0809305
S1131D70450666E372E880E090E0D5CF089581E0FF
S1131D80809346060895CF92DF92EF92FF92CF930D
S1131D90DF93EC018FEF93E0BC016C1B7D0B072EEE
S1131DA0000C880B990BC9D220E030E040E251E4EA
S1131DB095D36B017C01BE01DD0F880B990BBDD25D
S1131DC09B01AC01C701B6011DD2DF91CF91FF90F9
S1131DD0EF90DF90CF9008957F928F929F92AF9271
S1131DE0BF92CF92DF92EF92FF920F931F93CF9304
S1131DF0DF93812C912C540100E010E00F2EF3E2CC
S1131E00CF2EF0E2DF2EF02D6894772477F8C2E726
S1131E10D2E20F2EF8E2EF2EF0E2FF2EF02D1F9308
S1131E200F93DF92CF921F927F92DF93CF93FBD4D5
S1131E3020E030E248E060E0CE0188DE7FDF9F935F
S1131E408F93FF92EF921F927F92DF93CF93EBD405
S1131E5020E030E240E160E0CE0178DE6FDF93DF26
S1131E609B01AC01C501B40169D14B015C016BE07C
S1131E707BE882E090E057DF0F5F1F4F8DB79EB77E
S1131E8040968DBF9EBF0233110509F0C8CF20E0F4
S1131E9030E048E452E4C501B401B4D12EEA37E499
S1131EA04DE151E4AFD1DF91CF911F910F91FF909C
S1131EB0EF90DF90CF90BF90AF909F908F907F90E6
S1131EC00895CF92DF92EF92FF92CF93DF93C12CCC
S1131ED0D12C7601C0E0D0E031DF009711F42197D6
S1131EE00DC051DF9B01AC01C701B60127D16B01C5
S1131EF07C016BE171E480E090E015DF2196C53050
S1131F00D10554F320E030E040EA50E4C701B601C3
S1131F1079D1DF91CF91FF90EF90DF90CF9008952A
S1131F20CF93DF93EA019AD22C813D814E815F8168
S1131F3004D1288539854A855B8564D12881398116
S1131F404A815B81FBD09B01AC0160E070E080E2E0
S1131F5091E427D3BFD1CB01DF91CF910895CF93E3
S1131F60DF93CDB7DEB72C97CDBFDEBF3FDE0E9437
S1131F7025060E942803BE016F5F7F4F80E492E034
S1131F8072DBAE01485F5F4F61E080E492E0EFDB1B
S1131F909A818B818F7880618B83892F817E8A835C
S1131FA01C8282E08D8311E0188780E48987BE015A
S1131FB06F5F7F4F80E492E0F0DAAE01485F5F4FDD
S1131FC061E080E492E088DB80E492E00E94FB061A
S1131FD087E08093A200789480E180938506109333
S1131FE0410620E030E240E060E080E390E2AEDDD4
S1131FF0F3DE609307207093082080930920909368
S11320000A20612C6894772471F80F2EFFE38F2E39
S1132010F0E29F2EF02D6894FF24F7F802E712E215
S11320200F2EFBE4AF2EF0E2BF2EF02D0F2EF9E5BC
S1132030CF2EF0E2DF2EF02D0F2EF8E22F2EF0E25D
S11320403F2EF02D8FB78983F8949981F301808115
S1132050886080839FBF0E9412038823E1F30E945B
S1132060770388872EDF2091072030910820409144
S1132070092050910A20C6D04BE050E251DF582E7F
S1132080E92E1FDF2091072030910820409109207C
S113209050910A20B7D047E150E242DF482E9C8796
S11320A08885282F082E000C330B3F938F939F9223
S11320B08F921F92FF921F930F93B5D320E030E2CB
S11320C040E060E0C80142DDEF925F92BF92AF92C0
S11320D01F92FF921F930F93A6D320E030E248E0B3
S11320E060E0C80133DDFC85FF934F92DF92CF920D
S11320F01F92FF921F930F9396D320E030E240E1AA
S113210060E0C80123DD1ADE9F938F933F922F92E4
S11321101F92FF921F930F9386D3CDBFDEBF20E0A3
S113212030E248E160E0C80111DD8885652D7E2D2F
S1132130082E000C990B17DE85CF5058BB27AA2711
S11321400ED04DC13ED130F043D120F031F49F3F49
S113215011F41EF433C10EF4E095E7FB29C1E92F15
S11321604FD180F3BA17620773078407950718F0F5
S113217071F49EF567C10EF4E0950B2EBA2FA02DD5
S11321800B01B90190010C01CA01A0011124FF2720
S1132190591B99F0593F50F4503E68F11A16F0401B
S11321A0A22F232F342F4427585FF3CF469537951A
S11321B02795A795F0405395C9F77EF41F16BA0BDF
S11321C0620B730B840BBAF09150A1F0FF0FBB1F8D
S11321D0661F771F881FC2F70EC0BA0F621F731FD6
S11321E0841F48F4879577956795B795F7959E3F33
S11321F008F0B3CF9395880F08F09927EE0F9795C1
S1132200879508950CD0EBC0E3D040F0DAD030F0DD
S113221021F45F3F19F0CCC0511115C1CFC0F0D0EB
S113222098F39923C9F35523B1F3951B550BBB2799
S1132230AA2762177307840738F09F5F5F4F220F46
S1132240331F441FAA1FA9F333D00E2E3AF0E0E83F
S113225030D091505040E695001CCAF729D0FE2F8B
S113226027D0660F771F881FBB1F2617370748071D
S1132270AB07B0E809F0BB0B802DBF01FF279358D3
S11322805F4F2AF09E3F510568F092C0DCC05F3F6B
S1132290ECF3983EDCF3869577956795B795F795BB
S11322A09F5FC9F7880F911D9695879597F90895B3
S11322B0E1E0660F771F881FBB1F6217730784074F
S11322C0BA0720F0621B730B840BBA0BEE1F88F75E
S11322D0E095089504D06894B111B5C0089598D0DC
S11322E088F09F5790F0B92F9927B751A0F0D1F0FB
S11322F0660F771F881F991F1AF0BA95C9F712C085
S1132300B13081F09FD0B1E008959CC0672F782F41
S11323108827B85F39F0B93FCCF3869577956795F0
S1132320B395D9F73EF490958095709561957F4F5C
S11323308F4F9F4F0895E89409C097FB3EF4909502
S11323408095709561957F4F8F4F9F4F9923A9F08A
S1132350F92F96E9BB279395F69587957795679519
S1132360B795F111F8CFFAF4BB0F11F460FF1BC05D
S11323706F5F7F4F8F4F9F4F16C0882311F096E9F0
S113238011C0772321F09EE8872F762F05C066239E
S113239071F096E8862F70E060E02AF09A95660F57
S11323A0771F881FDAF7880F9695879597F9089510
S11323B097F99F6780E870E060E008959FEF80ECF4
S11323C0089500240A941616170618060906089597
S11323D000240A9412161306140605060895092EFD
S11323E00394000C11F4882352F0BB0F40F4BF2B6C
S11323F011F460FF04C06F5F7F4F8F4F9F4F0895AC
S113240057FD9058440F551F59F05F3F71F04795A1
S1132410880F97FB991F61F09F3F79F08795089586
S1132420121613061406551FF2CF4695F1DF08C0A5
S1132430161617061806991FF1CF869571056105C2
S113244008940895E894BB2766277727CB0197F96A
S113245008950EF023C1B2CF6894AACFD9DFC8F390
S11324609923D1F3C6F3DF93CF931F930F93FF9276
S1132470C92FDD2788232AF02197660F771F881F2D
S1132480DAF720E030E040E85FEB9FE3883920F0A2
S1132490803E30F021968F7751DEECEFF1E003C0FF
S11324A04DDEE9E2F2E008D18B01BE01EC01FB2E26
S11324B06F5771097595771F880B990B3EDF28E1DB
S11324C032E741E35FE316D0AF2D9801AE01FF90F0
S11324D00F911F91CF91DF9142DE81CF0BD07FCF3F
S11324E070DF28F075DF18F0952309F061CF66CF0F
S11324F01124A9CF85DFA0F3959FD1F3950F50E068
S1132500551F629FF001729FBB27F00DB11D639FA1
S1132510AA27F00DB11DAA1F649F6627B00DA11D47
S1132520661F829F2227B00DA11D621F739FB00DED
S1132530A11D621F839FA00D611D221F749F33275D
S1132540A00D611D231F849F600D211D822F762FF6
S11325506A2F11249F5750408AF0E1F088234AF0F3
S1132560EE0FFF1FBB1F661F771F881F915050403F
S1132570A9F79E3F510570F01BCF65CF5F3FECF389
S1132580983EDCF3869577956795B795F795E7952B
S11325909F5FC1F7FE2B880F911D9695879597F93C
S11325A00895FA01EE0FFF1F30962105310599F1C8
S11325B06115710561F48038BFE39B0749F16894A4
S11325C09038810561F08038BFEF9B0741F0992373
S11325D042F5FF3FE1053105210511F1E894089426
S11325E0E795D901AA2329F4AB2FBE2FF85FD0F3C6
S11325F010C0FF5F70F4A695E0F7F73950F019F0BA
S1132600FF3A38F49F779F930CD00F9007FC9058B3
S113261008953EF0D3CE60E070E080E89FE3089533
S11326204FE79F775F934F933F932F9317DF2F913C
S11326303F914F915F9152DF05C019F40EF0B8CE6F
S113264001CFBCCEE5DEC8F39638C0F707F80F9289
S1132650E8942BE33AEA48EB5FE74EDF0F920F92E0
S11326600F924DB75EB70F9289D0E6E5F2E024D021
S11326704F915F91EF91FF91E595EE1FFF1F49F098
S1132680FE57E0684427EE0F441FFA95E1F74195A1
S1132690550B40D00F9007FE34C008959F3F31F092
S11326A0915020F4879577956795B795880F911D7C
S11326B09695879597F90895DF93CF931F930F937A
S11326C0FF92EF92DF927B018C01689405C0DA2EB1
S11326D0EF0110DFFE01E894A59125913591459114
S11326E05591AEF3EF013BDDFE019701A801DA94A9
S11326F079F7DF90EF90FF900F911F91CF91DF91C9
S113270008959B01AC0160E070E080E89FE37ACD1E
S11327104FCEC4CF7DDEE8F39923D9F3940F511D36
S1132720BBF39150504094F059F0882332F0660F77
S1132730771F881F91505040C1F79E3F510544F7C1
S1132740880F911D9695879597F908955F3FACF092
S1132750983E9CF0BB27869577956795B79508F4C6
S1132760B1609395C1F7BB0F58F711F460FFE8CF40
S11327706F5F7F4F8F4F9F4FE3CF65CEFA01DC0130
S1132780AA0FBB1F9B01AC01BF5728F42227332794
S1132790442750781FC0B75188F4AB2F00244695C6
S11327A037952795011CA395D2F3002069F0220FD9
S11327B0331F441FB395DAF30DD0BFCC61307105DC
S11327C0A0E88A07B94630F49B01AC016627772755
S11327D088279078309621F0208331834283538375
S11327E00895A1E21A2EAA1BBB1BFD010DC0AA1F4E
S11327F0BB1FEE1FFF1FA217B307E407F50720F066
S1132800A21BB30BE40BF50B661F771F881F991FE0
S11328101A9469F760957095809590959B01AC0129
S1132820BD01CF0108950F931F93CF93DF93CDB7CD
S1132830DEB72E97CDBFDEBF0E891F89888D998D97
S113284026E02C8309831A8397FF02C080E090E876
S113285001978D839E83AE01445E5F4F6A8D7B8DAD
S1132860CE01019616D04D815E8157FD0AC02F819D
S11328703885421753070CF49A01F801E20FF31F4D
S113288010822E96CDBFDEBFDF91CF911F910F91A5
S113289008952F923F924F925F926F927F928F9200
S11328A09F92AF92BF92CF92DF92EF92FF920F93DB
S11328B01F93CF93DF93CDB7DEB72B97CDBFDEBF8A
S11328C06C017B018A01FC0116821782838181FFDE
S11328D0BFC1CE0101963C01F6019381F70193FD3E
S11328E0859193FF81917F01882309F4ADC18532DD
S11328F039F493FD859193FF81917F01853221F411
S1132900B60190E0D3D1E8CF912C212C312CFFE1FA
S1132910F315D8F08B3279F038F4803279F08332C1
S1132920A1F4232D20611DC08D3261F0803369F440
S1132930232D216016C0832D8260382EE32DE460A0
S11329403E2E2AC0F32DF8601DC037FC2DC020EDAB
S1132950280F2A3040F08E32B9F436FC75C1232D8D
S11329602064322E19C036FE06C08AE0989E200DDF
S11329701124922E11C0EAE02E9E200D1124222E45
S1132980F32DF0623F2E08C08C3621F4832D80682D
S1132990382E02C0883641F4F70193FD859193FFE8
S11329A081917F018111B3CF982F9F7D95549330EE
S11329B028F40C5F1F4F9FE399830DC0833631F0D9
S11329C0833771F0833509F055C020C0F801808148
S11329D089830E5F1F4F88248394912C530112C066
S11329E02801F2E04F0E511CF801A080B18036FEA0
S11329F003C0692D70E002C06FEF7FEFC5014BD1BA
S1132A004C018201F32DFF773F2E15C0280122E0EF
S1132A10420E511CF801A080B18036FE03C0692D1E
S1132A2070E002C06FEF7FEFC5012AD14C01F32D96
S1132A30F0683F2E820133FC19C0822D90E0881685
S1132A409906A0F4B60180E290E030D12A94F5CF43
S1132A50F50137FC859137FE81915F01B60190E065
S1132A6025D121102A9421E0821A9108811491041D
S1132A7079F7E1C0843611F0893639F5F80137FE6B
S1132A8007C060817181828193810C5F1F4F08C0F0
S1132A9060817181072E000C880B990B0E5F1F4F0C
S1132AA0F32DFF763F2E97FF09C090958095709582
S1132AB061957F4F8F4F9F4FF0683F2E2AE030E0A3
S1132AC0A30130D1882E861844C0853731F4232DD4
S1132AD02F7EB22E2AE030E025C0932D997FB92EA7
S1132AE08F36C1F018F4883579F0AEC0803719F00C
S1132AF0883721F0A9C0E92FE061BE2EB4FE0DC0D5
S1132B00FB2DF460BF2E09C034FE0AC0292F2660B5
S1132B10B22E06C028E030E005C020E130E002C05B
S1132B2020E132E0F801B7FE07C060817181828143
S1132B3093810C5F1F4F06C06081718180E090E03B
S1132B400E5F1F4FA301EED0882E8618FB2DFF7752
S1132B503F2E36FE0DC0232D2E7FA22E891458F44D
S1132B6034FE0BC032FC09C0832D8E7EA82E05C016
S1132B70B82CA32C03C0B82C01C0B92CA4FE0FC0E0
S1132B80FE01E80DF11D8081803321F49A2D997E98
S1132B90A92E09C0A2FE06C0B394B39404C08A2D22
S1132BA0867809F0B394A3FC10C0A0FE06C0B2144A
S1132BB080F4280C922C9B180DC0B21458F4B60162
S1132BC080E290E073D0B394F8CFB21418F42B18C9
S1132BD002C0982C212CA4FE0FC0B60180E390E023
S1132BE065D0A2FE16C0A1FC03C088E790E002C035
S1132BF088E590E0B6010CC08A2D867851F0A1FEDC
S1132C0002C08BE201C080E2A7FC8DE2B60190E035
S1132C104DD0891430F4B60180E390E047D09A9403
S1132C20F8CF8A94F301E80DF11D8081B60190E09C
S1132C303DD08110F6CF222009F44ECEB60180E2B9
S1132C4090E034D02A94F7CFF6018681978102C0B0
S1132C508FEF9FEF2B96CDBFDEBFDF91CF911F91FA
S1132C600F91FF90EF90DF90CF90BF90AF909F9027
S1132C708F907F906F905F904F903F902F9008952A
S1132C80FC010590615070400110D8F78095909533
S1132C908E0F9F1F0895FC01615070400190011038
S1132CA0D8F7809590958E0F9F1F08950F931F93CB
S1132CB0CF93DF93FB01238121FD03C08FEF9FEFAF
S1132CC02CC022FF16C046815781248135814217CA
S1132CD0530744F4A081B1819D012F5F3F4F2083AE
S1132CE031838C93268137812F5F3F4F268337832F
S1132CF014C08B01EC01FB010084F185E02D1995D2
S1132D00892BE1F6D80116968D919C91179701961F
S1132D1016968D939C931797CE01DF91CF911F91B7
S1132D200F910895FA01AA27283051F1203181F139
S1132D30E8946F936E7F6E5F7F4F8F4F9F4FAF4FBF
S1132D40B1E03ED0B4E03CD0670F781F891F9A1FD2
S1132D50A11D680F791F8A1F911DA11D6A0F711D86
S1132D60811D911DA11D20D009F468943F912AE092
S1132D70269F11243019305D3193DEF6CF0108957A
S1132D80462F4770405D4193B3E00FD0C9F7F6CFAB
S1132D90462F4F70405D4A3318F0495D31FD405273
S1132DA0419302D0A9F7EACFB4E0A6959795879509
S1132DB077956795BA95C9F70097610571050895E8
S1132DC09B01AC010A2E0694579547953795279594
S1132DD0BA95C9F7620F731F841F951FA01D08952C
S1072DE0F894FFCF91
S1132DE4007E020607207D00002041333313401483
S1132DF4AE073FF628DCBE33331340CDCC4C3E66DD
S1132E0466E6BE693D2564007261773A2025640054
S1132E1443616C6962726174696E672E2E2E00546C
S1132E24656D7072203A2025336400536D6F6B65B1
S1132E343A2025336470706D004C50473A20253392
S1092E446470706D0000D3
S9030000FC
